S016000077656967682D7363616C652D316B2E73726563FC
S11300002BC032C031C030C02FC02EC02DC02CC078
S11300102BC02AC029C028C027C026C025C024C0A0
S113002023C022C021C020C01FC01EC01DC01CC0D0
S11300301BC01AC0206B6720202020200020202015
S113004020202020200056312E3020202020005354
S113005063616C652020200011241FBECFEFD2E025
S1130060DEBFCDBFB7D08DC1CBCF449A81E38A9593
S1130070F1F700004498089598B182958F709827FD
S11300809F7096B9F2CF8A3010F4805D0895803164
S113009010F4895C08958FE308950F931F93CF9311
S11300A0DF93EA018901843058F49AE09C9FA0010F
S11300B09D9F500D1124215031098F5FEEDFBC014B
S11300C080E06C177D0720F08F5F6C1B7D0BF9CFF0
S11300D0805DF8018083CB01DF91CF911F910F9157
S11300E00895CF93C82F459AC7DF8C2F8295807FC0
S11300F0C3DF81E78A95F1F70000CF910895CF938C
S1130100C82F4598B9DF8C2F8295807FB5DF87E6AD
S11301108A95F1F70000CF91089581E0F0DF86E63B
S11301209EE00197F1F700000895613021F06230FC
S113013031F490E401C090E08058890FE0CF089535
S1130140D0CFCF93DF93EC018991882311F0C9DFDD
S1130150FBCFDF91CF910895CF93DF93EC01FE01A4
S11301608491882319F0BDDF2196F9CFDF91CF91D7
S11301700895FC0118992CC098E140E050E0BA01C0
S1130180299A82E08A95F1F700C02998440F551FF7
S1130190661F771F1899416082E08A95F1F700C0C5
S11301A0915071F767FD7F6F299A82E08A95F1F784
S11301B000C0299882E08A95F1F700C0440F551FCA
S11301C0661F771F408351836283738381E00895A0
S11301D080E00895CF93DF93CDB7DEB72E970FB6A7
S11301E0F894DEBF0FBECDBF82E084B98FE387B938
S11301F082E88AB98FEF9BE60197F1F700C000000F
S113020080E33ADF8FEF93E20197F1F700C000003B
S11302102CDF83E397E00197F1F727DF83E397E08F
S11302200197F1F780E228DF8FEF93E20197F1F76E
S113023000C0000088E263DF8CE061DF86E05FDFFE
S11302406CDF2998219A209861E080E06EDF8FE4CA
S113025090E082DF62E080E068DF86E490E07CDFAB
S1130260812C912C540110E0CE010B9682DF88235F
S113027049F01F5F8B859C85AD85BE85880E991ED0
S1130280AA1EBB1E143184F3B594A7949794879443
S113029061E080E04ADF8DE390E05EDF62E080E0D1
S11302A044DF84E390E058DFC12CD12C7601612C2B
S11302B00EE210E25DE2752ECE010B965ADF882322
S11302C0D9F363948B859C85AD85BE85C80ED91EF4
S11302D0EA1EFB1E99E096157CF7D701C601881922
S11302E09909AA09BB09292F3A2F4B2F552747FDF6
S11302F05A95A7E1B5E12FD0BB2797FDB095AB2F59
S1130300FC0197FD02C0198305C07982EE27FF27FF
S1130310E81BF90B9E012A5F3F4F41E050E0BF010B
S113032080E0BBDE8D818F838C818E830D83188664
S11303308A81803329F41A838B81803309F41B83E7
S113034061E081E0F2DECE010196FBDEC12CD12C0E
S11303507601612CB1CF09D0A59F900DB49F900D6B
S1130360A49F800D911D11240895A29FB001B39FF5
S1130370C001A39F01D0B29F700D811D1124911D56
S10903800895F894FFCF7C
S9030000FC
